S028000052414D436F646556325F4D433133323234565F496E7465726E616C5350495F4C452E6D6F74BD
S111000031005900AD00C90185028702890252
S1130010064B1860521E10024906490E0143802007
S1130020084398601869C007FCD5704700C0008079
S113003050680021018001228270C17002714271F6
S11300408171C271027241728272026141611F2127
S113005081611103C1617047F8B50E005568D0681D
S1130060116940185469746000273760844902227A
S11300708A602022202103021B0AC0208004184326
S1130080FFF7C6FF082200210020FFF7C1FF7C48CC
S113009000680006000E28706D1C641EF2D17848BA
S11300A003218160012181607760F1BDF2B582B0E6
S11300B00800002101605668D068116940180702E1
S11300C03F0A5569029845606D480121816001919C
S11300D010220821A020C004FFF79AFF6848006896
S11300E00006000E00900C2108420FD008220821BF
S11300F0A020C005FFF78CFF102210210098432395
S113010003401B0408051843FFF782FF0822082157
S1130110C020C004FFF77CFF3078000274780443E9
S1130120574802218160019800280ED02022202106
S1130130AD2000063843FFF76BFF10221021200486
S1130140FFF766FF0020019007E018221821230220
S1130150AD2000061843FFF75BFF49480321816087
S113016001218160B61CAD1E029845601022082151
S1130170A020C004FFF74CFF414800680006000EB1
S1130180C007F3D4002DC7D108220821C805FFF702
S11301903FFF10220821A020C004FFF739FF384890
S11301A004682406240E08220821A020C005FFF7B5
S11301B02FFF102210210C202043030408051843AC
S11301C0FFF726FF03B0F0BDF8B5002008602C4807
S11301D0012181605569D06811694018040BA0277A
S11301E0FF04102208213800FFF712FF244E306864
S11301F00006000E00900C2108420ED008220821AF
S11302003801FFF705FF1022102100984323034013
S11302101B0408051843FFF7FBFE08220821C02031
S1130220C004FFF7F5FE20222021200303021B0A4D
S113023008061843FFF7ECFE102208213800FFF7E8
S1130240E7FE30680006000EC007F5D4641C6D1E7E
S1130250E3D1102208213800FFF7DAFE34682406BF
S1130260240E082208213801FFF7D2FE10221021A3
S11302700C202043030408051843FFF7C9FEF1BD11
S10D028004C0008070477047704707
S9030000FC
